:100000000DC0D9C0FDCFFCCFFBCFFACFF9CF79C25D
:10001000F7CFF6CFF5CFF4CFF3CFE5C00FED0DBF9F
:10002000FF24C0E6D0E0F992C03EE9F70FE702BB3B
:1000300002E001BB00EE08BB0FE107BB09E110E0E5
:1000400012B909B908E90AB900E810E01BBD0ABDF8
:1000500019BD08BD01EA0FBD01E00EBD02E006BFFB
:1000600002E000BF03E003BF01E009BF02E005BFFB
:1000700000E40BBF91E000E06CD003E08AD0EEE436
:10008000F5E0D0D1E4E4F5E0CDD1B1D13D91313608
:1000900008F030523032B4F33B3209F46CC03D32D8
:1000A00009F469C03F3379F03D3489F03335C1F04C
:1000B0003035C9F0353479F0323589F13735B9F159
:1000C000E8E4F5E002C0EAEAF5E0ACD1DBCFB0D17C
:1000D000B9F35FD0D7CFACD199F300FB90F9D2CF71
:1000E000C0E7D0E009C0A4D159F3083048F7000FA9
:1000F000C02FDD27C05ADF4F9BD110F359F40AE01F
:10010000E6D108811981C0D10AE3E1D170D190D143
:10011000B8F221F0F894198308837894B3CF88D18A
:1001200079F2083068F6F89414D07894ABCF80D187
:1001300039F2083028F616D0E199FECF3EBB339550
:1001400009910DBBF894E29AE19A78941A95A1F777
:1001500099CF08D03EBB3395E09A0DB309931A9519
:10016000C9F7089510E13327015010F0310FFCCF8B
:10017000C0E6D0E00895632F5BD109F4A1CFF894D5
:100180006D3219F0800E911E02C0801A910A789487
:1001900079CFF89400937A00C0E7D0E0F992C8379D
:1001A000E9F7AA24BB248824992477247894C0985A
:1001B000C198C29A08951F930F931FB7869B08C0DA
:1001C00000916C00700E00916D00801E9F1C07C096
:1001D00000916C00701A00916D00800A9F081FBF8B
:1001E0000F911F9118950F92FF93EF930FB6EE2D7D
:1001F000E0B2E294F1E0E1FCEF26EE19E37089F061
:10020000E33039F0E13041F0ED2DFD2DEE0FF595A5
:1002100006C0EFEFFFEF02C0E1E0F0E0DE2EAE0E31
:10022000BF1ECA9409F0BCC0E3E5CE2E78941F929D
:100230000F923F922F921F930F933F932F935F93B1
:100240004F936F93DF93CF93C0E6D0E02E883F8823
:10025000F8942A183B08BF8AAE8A78943094219487
:1002600009F433940A8D033041F00888198802306C
:1002700011F1013009F46EC073C0F89404010A183A
:100280001B08789400E21EE4001611060CF08DC0E5
:1002900000EE11EB001611060CF487C008811981DD
:1002A000001611063CF41095019509F413950016FB
:1002B00011060CF4080181012A813B817CD0021ACD
:1002C000130A80012C813D8176D0F9010A891B89AE
:1002D0002E813F8170D0E20FF31F80012C893D8970
:1002E000021B130B2E853F8566D0E20FF31F1D8A7C
:1002F0000C8A9F7928853985E217F30714F0F901F4
:10030000906421953095E217F30714F4F901906297
:1003100011201AF096FD09C002C095FD06C00A8999
:100320001B89000D111D1B8B0A8B092F0076088D70
:10033000198D21F0C19A0D5F1F4F04C0C198015063
:10034000104038F0198F088F24EF31E0021713079F
:1003500060F50F0181012A853B852DD0020E131E09
:1003600000EF10E0001611062CF400E11FEF00165C
:1003700011060CF408011594079400E8001D10E81C
:1003800010190ABD18BDCF91DF916F914F915F9108
:100390002F913F910F911F912F903F900F901F90A1
:1003A0000FBEEF91FF910F90189500E0F2DEC09A1A
:1003B00000241124D5CFE89411232AF468941095D1
:1003C000019509F41395441B550B61E110F4400F9E
:1003D000511F57954795379527956A95B9F7232F5C
:1003E000342F26F43095219509F433950895ADE81E
:1003F000B0E030E070D0F1F30C930D3019F4ADE8BB
:10040000B0E063C0083031F43030A1F35ED0119712
:100410003A95F0CF003270F3333161F356D0119634
:100420003395E8CF0591002309F4089550D0FACF11
:10043000E894002711273D91303210F1E1F33D326D
:1004400011F468943D91313298F0305370F03A30A5
:1004500060F441E1222726951795079508F4265F59
:100460004A95C9F7030F1F1DEDCF089418940895FE
:10047000119726F41095019509F413958894089521
:10048000119788941894089550E217FF05C01095AD
:10049000019509F413955DE200240394222740E1BD
:1004A000000F111F221F2A3010F02A5003954A9581
:1004B000B9F7205D2F930F151F0579F7052F07D08A
:1004C0000F9105D00A94E1F7089590FF08955D9B80
:1004D000FECF0CB908951F93DF93CF93CBE7D0E005
:1004E000F89418810981101739F0C10F0A81C11BD6
:1004F00013951F70188398947894CF91DF911F9172
:1005000008950F930FB72F932CB1579878941F939A
:100510000F93DF93CF93CBE7D0E008811981139538
:100520001F70101729F019831A951F70C10F2A83A5
:10053000CF91DF910F911F912F910FBF0F91F894E1
:10054000579A18950D0A25000A3F3F3F00000D0AF3
:10055000534D433341202D20536572766F204D6FEC
:10056000746F7220436F6E74726F6C6C6572204B87
:100570006F5A6F3A312E3020284D6F64653A332020
:100580002C2044746167202C20536572766F20689C
:100590006962612069646F3A3530306D7329283F94
:1005A0003A68656C70290D0A00000D0A6D3C6D6F8C
:1005B000643E202D20736572766F206D6F64650D2B
:1005C0000A653C6D6F643E202D206563686F206D69
:1005D0006F64650D0A733C76616C3E202D20737547
:1005E0006220636D640D0A7B2B7C2D7D3C737470DF
:1005F0003E202D207374657020636D640D0A703C7D
:100600007061723E205B3C76616C3E5D202D206502
:1006100078616D696E652F6368616E6765207061D2
:10062000726D730D0A773C626E6B3E202D207361F4
:100630007665207061726D730D0A723C626E6B3E5E
:10064000202D206C6F6164207061726D7300FFFF5C
:100800009001A00F40066400B400580200010100EE
:00000001FF
